:020000020000FC
:1000000056C028E0C49A16B31078E1F307FDC69AEB
:1000100007FFC698000000000000C49816B31078CF
:10002000E9F7000F2A9571F70895112422242A94E4
:10003000F1F71A94E1F73A95D1F708958A9A9298D0
:1000400032E0F3DF30E033BF32BF32E033BF8A98B3
:1000500032B73831E8F330E033BF32BF32E033BF7C
:1000600042B74F3F11F0829BFBCF30E033BF32BF2E
:10007000332D341B323010F0342E01C0432D469501
:100080004695089552E0C298C098C29A642F78E0CD
:10009000C09A60FDC19860FFC19A0000C09800003E
:1000A00066957A95A9F75A9589F7C2980895B89AEE
:1000B000BA9AB99ABC9ABE9ABF98C0DFE3DFFDCF67
:00000001FF
